:100000000C9439030C9461030C9461030C94610308
:100010000C9461030C9461030C9461030C946103D0
:100020000C9461030C9461030C9461030C94D81E2E
:100030000C9461030C9461030C9461030C946103B0
:100040000C94BD1F0C9461030C9461030C94610328
:100050000C9461030C9461030C9461030C94610390
:100060000C9461030C946103506F636B65742045BD
:100070006D70697265730080007B00517569740052
:10008000526573756D65000808FC848884A2D10AE6
:10009000044661696C656420746F206372656174E5
:1000A0006520756E697421004661696C6564207411
:1000B0006F20637265617465206275696C64696E36
:1000C0006721000808003C4299A5661800080860EE
:1000D000BCC299A5671D02FD00EC00E400DF0051E1
:1000E000756974004F7074696F6E73004D756C7430
:1000F00069706C617965722067616D650053696E26
:10010000676C6520706C617965722067616D650050
:1001100018180000000000FEFE00FEFE003E3E003B
:10012000FEFE00FEFE001E1E001E1E001E1E001E05
:100130001E001E1E001E1E001E1E001E1E001E1E75
:10014000001E1E001E1E001E1E00FEFE00FEFE0003
:100150003E3E00FEFE00FEFE00FE1818E700E7BD72
:1001600000BDE7FFE7BD00BD81FF81E700E7A50017
:10017000A5BDFFBDA500A5A500A5A500A5A500A539
:10018000A500A5A500A5A500A5A500A5E700E7BDBC
:1001900000BDE7FFE7BD00BD81FF8181188181249B
:1001A00081FFFFFF03030705070504050504050399
:1001B00006030207020201020203020E090E0E0DDF
:1001C0000E0E0F0E070507050307050F05070507A8
:1001D00006070102050200070202070002070200EB
:1001E00002070200070603060707020205050201CF
:1001F00002020402000502020500060705050705C4
:10020000020302020602000000000B0003000307C5
:10021000050704070105020507070400030000079E
:1002200005050700050005020702000C0002020296
:10023000000400040201070507050704010704057F
:100240000702030207040701070606010107070763
:1002500007030307000500000D0002050005050562
:100260000005020107030F09030603060707020240
:10027000050507070207070507030107050607022B
:10028000070507050404030702050704040703071D
:10029000070106070507070303070503070306040D
:1002A0000701010701070407030403070607050206
:1002B0000501060101070400070501020405070006
:1002C00002010208080800030006030607070202ED
:1002D00005050705020707050703010705060702CD
:1002E00007050705040403070205070404070307BD
:1002F00007010607050707030307050307030604AD
:1003000007010107010704070304030706070502A5
:1003100005010601010704020705000700050702A1
:1003200006020307050703053F213F1208120A10C2
:100330000A0E1C0E0C1E0C141A14161F161E131E69
:100340001E1B1E1E1F1E3F213F3A2F3A173D173F0F
:10035000213F181F02040A041F0E04040E1F0A1F67
:100360000A0E0E1F04110E2E252E2F2A2E262929A5
:10037000021F02081F08150E04040E150E15151B8A
:10038000151B040604040C04000000001700030001
:10039000031F0A1F16371A1904130A153A0003001F
:1003A000000E11110E000A040A040E0400300004AD
:1003B00004040010001804031F111F121F101D1544
:1003C0001711151F07041F17151D1F151D01011FEC
:1003D0001F151F17151F000A00003200040A110A1A
:1003E0000A0A110A040115020E11171E051E1F1517
:1003F0000A0E110A1F110E1F15111F05010E111DE6
:100400001F041F111F1108100F1F041B1F10101FA6
:10041000061F1E040F0E110E1F09060E112E1F05BA
:100420001A121509011F011F101F0F180F1F0C1F93
:100430001B041B031C03191513001F1103041811BF
:100440001F000201022020200001020C121E1F12B8
:100450000C0C12120C121F0C1A14041E05242A1E56
:100460001F021C141D1020201D1F0814111F101E18
:10047000041E1E021C0C120C3E0A040C123E1E042A
:100480000214160A020F120E101E0E100E1E081E67
:10049000120C1226281E322A26041E21001F0021BB
:1004A0001E040102013F213F0A4E6F205344206386
:1004B000617264206F720A6E6F204C4F4144455246
:1004C0002E4845580A0A153A45786974001D204699
:1004D0006C617368696E670A20206C6F6164657275
:1004E0002E2E2E0A0A444F4E2754205455524E2089
:1004F0004F464621000A0A153A49676E6F72650039
:100500006D560A0A504C45415345205455524E20D1
:100510004F464620004C4F572042415454455259B3
:1005200021200017534400161378001613140015E9
:1005300010200015201000540A03E181867F3E1828
:100540006D830F0F0E0183866033186DC3198F18EA
:1005500003C38E6033186DE330CF1803C39E60363B
:1005600030CDE360CF3006C79E7E3E30CDB360CF46
:10057000300CC6F6603330D9B660CF33CFCCF660DE
:1005800061B0DB1E60CF30D86CE6C061B0DB1E61AD
:100590008F19986CC6C063B19B0E330F0FB078C62D
:1005A000FF7E1F1B061E0F05008930080238024916
:1005B0007868140000F6E8DBCFC3B8AEA49B928A3B
:1005C000827B746E68625C57524E4945413E3A37B1
:1005D00034312E2C29272523211F1D1C1A191716EB
:1005E0001514131211100F0E0D0C0B0A0908070633
:1005F00045006801000005006801380100000500A1
:100600003801680100000E060A060101FF0301011E
:10061000F7030000000700020100000304060000C9
:1006200000000000000001020408102040800102C8
:100630000408102001020408102004040404040427
:100640000404020202020202030303030303000084
:1006500000002300260029000000000025002800DB
:100660002B0000000000240027002A007403BF03B1
:10067000C30311241FBECFEFD8E0DEBFCDBF11E012
:10068000A0E0B1E0ECE7F1E502C005900D92A035E5
:10069000B107D9F727E0A0E5B1E001C01D92A73A64
:1006A000B207E1F713E0C8E3D3E004C02197FE01ED
:1006B0000E942924C633D107C9F70E9463030C9412
:1006C000B1280C9400000E945E200E94460480E540
:1006D00091E00E94F51B68E670E080E591E00E94E1
:1006E000781B0E94B20EF7CF1092A1011092A001C8
:1006F00085E491E090939F0180939E01089580EEA0
:1007000091E00E94DB0887E890E09093DF018093FE
:10071000DE0182E08093DD011092DB011092DC01AA
:1007200086E28093D70184E18093D8010E9403057B
:1007300086E090E00E948006882349F042E067E767
:1007400070E080E591E00E94B3188111089580EE79
:1007500091E00E942F0C0E94B40681110E94C703F1
:100760000E940B058823E1F380EE91E00E940107CF
:1007700087ED91E00E941C050E94E303D9CF80EE33
:1007800091E00C94C40680EE91E00C94C506809133
:100790006605811117C081E0809366053091670579
:1007A000209168058091690580916A0580916B05AB
:1007B00080916C0580916D0580916E05832F922F3D
:1007C0000C94B925089520916705309168054091F2
:1007D000690550916A0560916B0570916C05809177
:1007E0006D0590916E05A1E00E941D242093670580
:1007F000309368054093690550936A0560936B05D3
:1008000070936C0580936D0590936E0508958F929B
:100810009F92AF92BF92CF92DF92EF92FF924B01E5
:100820005C0169017A010E94B425BC01990F880B13
:10083000990BC818D908EA08FB08A70196012F5F91
:100840003F4F4F4F5F4F0E94D123680D791D8A1D86
:100850009B1DFF90EF90DF90CF90BF90AF909F9047
:100860008F900895E4E0F5E01386128611861086D5
:1008700010821182128213821482158216821782CC
:100880003C9685E0E436F80779F7089510926705FD
:10089000109268051092690510926A0510926B0516
:1008A00010926C0510926D0510926E051092650500
:1008B0000E943204109264050895EF92FF920F9304
:1008C0001F93CF93DF93CDB7DEB72C970FB6F89475
:1008D000DEBF0FBECDBF49835A836B837C839E836B
:1008E000EF82F88609871A873C8769817A814F8170
:1008F0005885240F352F311D62177307C8F4860FF2
:10090000972F911D4817590798F46B817C81498571
:100910005A858C85840F952F911D6817790740F4AF
:100920002E81260F372F311D81E04217530708F023
:1009300080E081702C960FB6F894DEBF0FBECDBF5D
:10094000DF91CF911F910F91FF90EF90089550E0AC
:10095000480F511D87FD5A9557FD0CC0843554F43E
:1009600030E0260F311D67FD3A9537FD03C081E069
:1009700060330CF080E00895DC01643508F042C07B
:10098000403308F03FC090968C919097E62F062E4A
:10099000000CFF0B242F25952595259594E529021C
:1009A000E00DF11D1124E856FA4F2081342F3770E5
:1009B0008230A1F4822F90E0032E02C09595879596
:1009C0000A94E2F780958170882399F081E090E0A5
:1009D00001C0880F3A95EAF7822B13C08330A1F744
:1009E0001C968C916427062E000C770B682760FDFF
:1009F000EDCF81E090E001C0880F3A95EAF780954D
:100A00008223808308951092A40166E273E08EE948
:100A100091E00C941E1580E591E00E94FB1791E097
:100A2000811101C090E0892F0895FC01238142814A
:100A3000618180810C94A704EF920F931F93CF9351
:100A4000DF93EC010E9415058823E1F01091BE01AF
:100A500040E06E818EE991E00E9471102F8138850F
:100A6000ED800C81498168818EE991E00E94371404
:100A7000612F8EE991E0DF91CF911F910F91EF905F
:100A80000C946D10DF91CF911F910F91EF9008950D
:100A9000FC01849108950196FC01849108954CE332
:100AA000BC0180E591E00C94D3160F931F93CF9374
:100AB000DF938C01C091BC01D091BD01229740937E
:100AC000A7012093A8018EE991E00E941E1540E045
:100AD00061E08EE991E00E947110B8018EE991E029
:100AE0000E942722209749F0BE018EE991E0DF9114
:100AF000CF911F910F910C941E15DF91CF911F91F3
:100B00000F910895FF920F931F93CF93DF93D82FE8
:100B1000162FC42FF22E242F0E94A7048823C1F081
:100B20000091BE016F2D8EE991E00E946D102C2F77
:100B3000412F6D2F8EE991E00E94FE10602F8EE90B
:100B400091E0DF91CF911F910F91FF900C946D1068
:100B5000DF91CF911F910F91FF900895EF92FF9237
:100B60000F931F93CF93DF93C82FD62F142FF22EFE
:100B70000E94A7048823D1F0E090BE01602F8EE987
:100B800091E00E946D100F2D212F4D2F6C2F8EE9BB
:100B900091E00E94AD106E2D8EE991E0DF91CF9132
:100BA0001F910F91FF90EF900C946D10DF91CF91FA
:100BB0001F910F91FF90EF900895EF92FF920F9386
:100BC0001F93CF93DF93C82FD62F142FF22E0E949E
:100BD000A7048823D1F0E090BE01602F8EE991E058
:100BE0000E946D100F2D212F4D2F6C2F8EE991E05B
:100BF0000E94D5106E2D8EE991E0DF91CF911F916B
:100C00000F91FF90EF900C946D10DF91CF911F9199
:100C10000F91FF90EF900895CF92DF92FF920F9384
:100C20001F93CF93DF93CDB7DEB728970FB6F89415
:100C3000DEBF0FBECDBF6C0160E08EE991E00E9487
:100C40006D1005E024E540E060E08EE991E00E944F
:100C5000D510F60180811F928F9386E091E09F93DB
:100C60008F931F9288E0F82EFF928E010F5F1F4F27
:100C70001F930F930E94C42521E044E064EA71E0D1
:100C8000C8010E945505F60181811F928F938BE068
:100C900091E09F938F931F92FF921F930F930E9457
:100CA000C42521E048E164EA71E0C8010E945505CD
:100CB000F60182811F928F9380E191E09F938F9341
:100CC0001F92FF921F930F930E94C42521E040E3DF
:100CD00064EA71E0C8010E9455050FB6F894DEBFC2
:100CE0000FBECDBF28960FB6F894DEBF0FBECDBFA6
:100CF000DF91CF911F910F91FF90DF90CF900895DA
:100D0000682F8AE591E00E94CC0F91E0811101C02B
:100D100090E0892F0895CF93C62F682F8AE591E040
:100D20000E94EB0F91E0C81708F090E0892FCF9157
:100D3000089560E00C948B0681E090E00E94990693
:100D4000811110C083E090E00E94990681110AC0D1
:100D500090E080E00E949906811104C082E090E05A
:100D60000C94990681E008950E949C0681110AC0A6
:100D700084E090E00E949906811104C085E090E033
:100D80000C94990681E00895089508950F931F9398
:100D9000CF93DF93CDB7DEB728970FB6F894DEBFB9
:100DA0000FBECDBF162F00E028E044E56BE280E0E7
:100DB0000E94DD051F921F9385E191E09F938F9321
:100DC0001F9288E08F938E010F5F1F4F1F930F9329
:100DD0000E94C4252CE244E064EA71E0C8010E944C
:100DE00055050FB6F894DEBF0FBECDBF28960FB6DF
:100DF000F894DEBF0FBECDBFDF91CF911F910F9151
:100E000008956F927F928F929F92AF92BF92CF92EE
:100E1000DF92EF92FF920F931F93CF93DF93EC013A
:100E20004C0180E1881A8EEF980A8E017E01E0EF76
:100E3000EE1AECEFFE0A712C6E01FEEECF1AFCEFFB
:100E4000DF0A5E0187EEA81A8CEFB80AF4018781E9
:100E50008823D1F041E0F6018081918188159905C0
:100E600009F040E0B401C5010E94FA0EF40160846B
:100E7000662051F0711008C06481CE010E94C60640
:100E8000C4010E94ED0E762CF9E08F0E911C8E1499
:100E90009F04E1F64E0180E2881A8EEF980A5E0107
:100EA000E7EEAE1AECEFBE0AF801858D8823F1F06B
:100EB0006801F0E1CF0ED11C41E0F7018081918102
:100EC0008C159D0509F040E0B601C5010E946F0D2B
:100ED000F801668C662051F0711008C0608DCE015B
:100EE0000E94C606C6010E945F0E762C015F1F4F4E
:100EF00008151905C9F6CD5DDC4F4881442331F052
:100F000001E022E06CE284E40E94AE05DF91CF9123
:100F10001F910F91FF90EF90DF90CF90BF90AF9017
:100F20009F908F907F906F9008956F927F928F9295
:100F30009F92AF92BF92CF92DF92EF92FF920F9368
:100F40001F93CF93DF9300D000D000D0CDB7DEB792
:100F50004C015B013C0180EF681A8CEF780A640158
:100F6000E0E1CE1AEEEFDE0AF6018781882309F46C
:100F70005AC0808191819A838983828193819C83E5
:100F80008B83858196810E94EE0E8D83F60185818B
:100F900096810E94F40E8E83E980FA800B811C8179
:100FA0002D81382FF50140815181628173818481C7
:100FB00095810E945D048823B1F120E830E040E093
:100FC00050E060E070E0CB010E940704F5017183FE
:100FD000608320E830E040E050E060E070E0CB016A
:100FE0000E940704F50173836283809170058F5F0F
:100FF00080937005803108F4B2CF80E026960FB65A
:10100000F894DEBF0FBECDBFDF91CF911F910F913E
:10101000FF90EF90DF90CF90BF90AF909F908F9018
:101020007F906F900895F9E0CF0ED11CC614D704BD
:1010300009F09ACF1092700581E0E0CF8F929F92D5
:10104000AF92BF92CF92DF92EF92FF920F931F93D6
:10105000CF93DF9300D000D000D0CDB7DEB77C01B6
:101060004B0109831A832B833C834D835E83BE012E
:101070006F5F7F4F0E949507B82E8823A9F1670103
:101080008AEEC81A8CEFD80AF6018081803208F007
:101090003FC099E0A92E8701A89E000D111D1124C3
:1010A000F801EB50FE4F91828082359789819A81B9
:1010B0009183808332968B819C8191838083C4014C
:1010C0000E94EB0EF801EC50FE4F8083F601808108
:1010D000A89EE00CF11C1124F701E950FE4F91E0AD
:1010E00090838F5FF60180838B2D26960FB6F89440
:1010F000DEBF0FBECDBFDF91CF911F910F91FF904B
:10110000EF90DF90CF90BF90AF909F908F90089519
:10111000B12CEACFBF92CF92DF92EF92FF920F9362
:101120001F93CF93DF9300D000D000D0CDB7DEB7B0
:101130007C01862F09831A832B833C8367019BEEF6
:10114000C91A9CEFD90AF6019081903290F52FE0F0
:10115000B22E8701B99E000D111D1124F801618F77
:1011600029813A81318B208B2B813C81338B228BDF
:101170000E94180EF801808FF6018081F701B89E59
:10118000E00DF11D112491E0958F8F5FF6018083B2
:1011900081E026960FB6F894DEBF0FBECDBFDF917B
:1011A000CF911F910F91FF90EF90DF90CF90BF9064
:1011B000089580E0EECFEF92FF920F931F93CF93AD
:1011C000DF9300D000D000D0CDB7DEB77C01FC01AA
:1011D000EB5EFC4F1082319610828C01005F1C4F39
:1011E000D8011D921C92349711821082875E9C4F09
:1011F0000E945E0C0E94C20E0E943F0DF701E0515A
:10120000FE4FCF0129E0DF01322F1D923A95E9F719
:101210003996E017F107B9F7F70170962FE0DF0173
:10122000322F1D923A95E9F73F96E817F907B9F77B
:1012300089E1F701E05EFC4F808382E33196808391
:101240008BE43196808324E130E040E050E060E0C0
:1012500070E0CB010E9407047A83698324E130E0C7
:1012600040E050E060E070E0CB010E9407047C8326
:101270006B8390E080E00E94EE0E8D8390E080E032
:101280000E94F40E09811A812B813C814D81582FD7
:1012900070E060E0C7010E941E08811104C088EA66
:1012A00090E00E944F0528E330E040E050E060E32A
:1012B00070E080E090E00E9407047A83698328E36D
:1012C00030E040E050E060E370E080E090E00E94B9
:1012D00007047C836B8380E00E94690D8D8380E02E
:1012E0000E94120E09811A812B813C814D81582F59
:1012F00060E0C7010E948A08811110C081E990E076
:1013000026960FB6F894DEBF0FBECDBFDF91CF910A
:101310001F910F91FF90EF900C944F0526960FB6FA
:10132000F894DEBF0FBECDBFDF91CF911F910F911B
:10133000FF90EF900895CF93DF9300D000D000D0BE
:10134000CDB7DEB7FC01E55EFC4F2081318144E181
:1013500050E0421B530B875E9C4FFC0180819181C2
:1013600026E230E0281B390B3A8329835C834B83C8
:101370003A815C8168E078E080E090E026960FB6E4
:10138000F894DEBF0FBECDBFDF91CF9108952F92AD
:101390003F924F925F926F927F928F929F92AF9205
:1013A000BF92CF92DF92EF92FF920F931F93CF9352
:1013B000DF93CDB7DEB761970FB6F894DEBF0FBEEF
:1013C000CDBF8C012C0120E2421A2EEF520A7C0183
:1013D00088248A94982C5401312C212CF701858D76
:1013E0008823D9F1868D811138C0C8010E949B09DC
:1013F00029833A834B835C836D837E83F701C088A6
:10140000D18862887388818D0E94690DF701818D72
:101410000E94120E89819A81C81AD90A8B819C81F7
:10142000681A790ACC9CC001CD9C900D900D1124B6
:10143000669C9001679C300D300D1124820F931F24
:10144000B0E0A0E088159905AA05BB0530F41701A6
:10145000F0E12F0E311C4C015D012FE0E20EF11C7A
:10146000E414F50409F0BACF780130E1E31A3EEF55
:10147000F30AB801605F7C4F798B688B44244A94EF
:10148000542C32011F821886E4E0CE2ED12CE9863E
:10149000FA86F7018781882309F463C0808581116A
:1014A00060C0C8010E949B0929833A834B835C83F7
:1014B0006D837E83F7010190F081E02DFC87EB873F
:1014C000F7010280F381E02DFE87ED87F70185812A
:1014D00096810E94EE0E8F87F701858196810E948A
:1014E000F40E29813A81A601421B530B2B853C85C2
:1014F000420F531F6F85262F30E035952795420FF9
:10150000531F2B813C81F601E21BF30B9F016D857C
:101510007E85260F371F90E095958795280F391FF8
:10152000449FC001459F900D900D1124229FA00162
:10153000239F500D500D1124840F951FB0E0A0E0A3
:1015400084159505A605B70530F0D301C2017F814A
:101550007987E885EA872C013D01F985FF832A8593
:10156000288739E0E30EF11C688979896E157F05BB
:1015700009F08DCFD801A05FBC4FF801EE5EFC4FA3
:1015800084149504A604B70490F111961C921E923F
:101590007F8170838885818391E9891691E099061E
:1015A000A104B10458F021E9421621E05206610479
:1015B000710420F01D921C921182108261960FB668
:1015C000F894DEBF0FBECDBFDF91CF911F910F9179
:1015D000FF90EF90DF90CF90BF90AF909F908F9053
:1015E0007F906F905F904F903F902F90089511964D
:1015F0003C922E9211821082CFCF0F931F93CF93E4
:10160000DF93EC01FC01E850FE4F8C01885E9C4F9B
:1016100020812223D9F0FE01EE5EFC4F8081918172
:101620000E94ED0ECE0180529E4FF801268D22239E
:1016300091F0C05FDC4F888199810E945F0E009716
:1016400081F4DF91CF911F910F9108953996E8179A
:10165000F907F1F6E7CF015F1F4F8017910729F7D0
:10166000F0CF2CE240E364EA71E0DF91CF911F916B
:101670000F910C945505EF92FF920F931F93CF9308
:10168000DF9300D000D000D0CDB7DEB78C0184E06E
:1016900090E00E949906882341F0F801ED5DFC4F2F
:1016A0008081853010F48F5F808384E090E00E9419
:1016B0008006882309F444C0F801E05FFC4FA08154
:1016C000B181C8014096980120513E4F41E0A817D2
:1016D000B90719F41E964C931E970F96821793071D
:1016E000B1F7D801AE5EBC4F0D90BC91A02D21E0AA
:1016F000A817B90719F418962C93189709968E17FE
:101700009F07B1F785E090E00E948006882329F0CA
:1017100080916F05882309F465C085E090E00E9400
:101720008006811187C026960FB6F894DEBF0FBEE3
:10173000CDBFDF91CF911F910F91FF90EF90089552
:1017400065E084E090E00E948B068823C9F0F801F0
:1017500030E020E0868D882361F04FE0429FC00199
:10176000439F900D11244096800F911F0E947E0E82
:10177000C9CF2F5F3F4F3F962032310559F7C2CF77
:1017800065E085E090E00E948B06882321F080913F
:101790006F05882329F0F801ED5DFC4F1082B2CF70
:1017A000C80180529E4FF801168E3F96E817F90740
:1017B000D9F7F801E850FE4FC801885E9C4F1082AF
:1017C0003996E817F907D9F7D801A05FBC4F1196F1
:1017D0001C921E9212961D921C9281E080936F05BE
:1017E000808390CFF801E85EFC4F8081811120C09A
:1017F000C8010E949B0929833A834B835C836D83D4
:101800007E83780180E2E81A8EEFF80AF801868D6F
:10181000882341F04B815C8169817A81C8014096BF
:101820000E941A0E015F1F4F0E151F0579F77BCF1F
:10183000108279CF80916F05882309F474CF1092BC
:101840006F0526960FB6F894DEBF0FBECDBFDF91B1
:10185000CF911F910F91FF90EF900C94A50EEF92F6
:10186000FF920F931F93CF93DF93EC01875E9C4F02
:101870000E94A50CCE010E94C7098E01005F1F4F78
:101880007E0180E1E81A8EEFF80AC8010E94220E5C
:10189000015F1F4F0E151F05C1F7CE010E943B0BC4
:1018A000CE010E94FD0ACE01805E9C4FDF91CF9158
:1018B0001F910F91FF90EF900C940C06FC01118288
:1018C0001082138212821482158283E08683089527
:1018D000CF93DF93CDB7DEB72C970FB6F894DEBF6A
:1018E0000FBECDBF1C861B86FC0120813181620F9B
:1018F000731F78876F8382819381480F591F5A879E
:10190000498786E0FE013796DE01119601900D921F
:101910008A95E1F729813A814B815C816D817E81D5
:1019200080E090E02C960FB6F894DEBF0FBECDBFDE
:10193000DF91CF910895FC019081490FDB014C9319
:101940008281280F11962C930895CF93DF93EC0199
:101950008E818330D8F48F5F8E832C81888199812A
:10196000820F911D27FD9A9597FF80C099838883E8
:101970002D818A819B81820F911D27FD9A9597FF6A
:1019800079C09B838A83DF91CF9108951E820E9444
:101990009C06882369F190E080E00E9499068823E4
:1019A00029F08C8187FF47C08E5F8C8381E090E0B7
:1019B0000E949906882329F08D8187FF41C08E5FA0
:1019C0008D8383E090E00E949906882331F08D8119
:1019D00018160CF03AC082508D8382E090E00E948D
:1019E0009906882329F08C8118169CF582508C83E7
:1019F00090E080E00E94990681110BC082E090E0A7
:101A00000E949906811105C08C81181634F5815009
:101A10008C8381E090E00E94990681119ECF83E043
:101A200090E00E949906811198CF8D811816CCF410
:101A300081508D8392CF85300CF0B8CF8F5FB5CFBA
:101A400085300CF0BECF8F5FBBCF8C3F34F281501E
:101A5000C3CF8C3F6CF28150CACF8823D1F28F5F05
:101A6000D7CF882309F479CF8F5FE3CF198218820B
:101A70001C827ECF1B821A821D8285CF08951F9300
:101A8000CF93DF93CCE7D5E083EC90E098878F830A
:101A90000E9448058A8383EC90E00E944B058B836B
:101AA0001D821C8211E01E83C3E7D5E08DEC90E01F
:101AB00098878F830E9448058A838DEC90E00E946E
:101AC0004B058B831D821C821E83DF91CF911F915A
:101AD000089580918305909184050C944805BF92E8
:101AE000CF92DF92EF92FF920F931F93CF93DF93EA
:101AF00000D000D000D0CDB7DEB76C018B01B42E82
:101B0000FB018585882309F458C0848523E7E22EEC
:101B100025E0F22E811104C09CE7E92E95E0F92E14
:101B2000F8019285F70194831582882341F0809112
:101B30007205882321F081E0911182E08583F8010C
:101B40008385811106C0F7018581911146C08260AD
:101B50008583F8012281338140815181B701C6011B
:101B60000E949B0CC7010E941C05F8018685BB20C2
:101B7000B1F1811134C04281538160817181C6010C
:101B80000E94680C29833A834B835C83F80181852A
:101B90000E94690D6B817C816D5F7F4FE981FA81C5
:101BA00023E0482FCF0103960E94820580917105A2
:101BB0008F5F853070F58093710526960FB6F89487
:101BC000DEBF0FBECDBFDF91CF911F910F91FF9070
:101BD000EF90DF90CF90BF9008958160B9CF8823B8
:101BE00029F3F8014281538160817181C6010E940D
:101BF000680C29833A834B835C83F80181850E94BA
:101C0000690D6B817C816D5F7F4FE981FA8121E0F5
:101C1000C8CF109271058091720591E08927809359
:101C20007205CBCF80918305909184050C944B0570
:101C300089E10895FC01758364835783468381E0BD
:101C400084870895FC0184858823F9F020813181FF
:101C5000B901615071094481558146175707B0F4A5
:101C60007183608391E092871386982F228133815C
:101C7000B90161507109468157814617570790F4A1
:101C80007383628312861386848708952F5F3F4F84
:101C900090E02417350750F73183208391E0928735
:101CA0009387E3CF2F5F3F4F2417350730F43383FB
:101CB0002283128691E09387E7CF892FE5CF209189
:101CC0008505222329F0213079F090E080E0089505
:101CD000DC011996EC91B4E0EB9FF0011124E75C74
:101CE000FE4F808191810895DC011996EC91B4E05A
:101CF000EB9FF0011124EF5CFE4FF3CF209185059F
:101D0000222319F02130A9F00895DC011996EC91F5
:101D1000B4E0EB9FF0011124E75CFE4F0280F381F9
:101D2000E02D309781F421110FC081E0809385056B
:101D30000895DC011996EC91B4E0EB9FF0011124B9
:101D4000EF5CFE4FEBCF099408951092850508953E
:101D500020E1FC0111922A95E9F7BC0180E591E0B0
:101D60000C94501C43E067ED70E080E591E00E9428
:101D7000B318811106C080EE91E00E94A80E0C9469
:101D80007F030895CF93DF93CFE8D5E08AE591E014
:101D900098878F830E9448058A838AE591E00E9494
:101DA0004B058B831D821C8281E08E83C6E8D5E0C3
:101DB00080E191E098878F830E9448058A8380E1C3
:101DC00091E00E944B058B831D821C8283E08E83F1
:101DD000DF91CF91089584E6089508958091960546
:101DE000909197050C9448058091960590919705E0
:101DF0000C944B05BF92CF92DF92EF92FF920F931C
:101E00001F93CF93DF9300D000D000D0CDB7DEB7C3
:101E10006C017B01142FFB018781882331F1228122
:101E20003381408151814650510966E875E0C60111
:101E30000E949B0C86E895E00E941C05F701228118
:101E40003381408151816FE875E0C6010E949B0C8F
:101E50008FE895E00E941C05F7018085112311F0A1
:101E6000882399F001E0811111C026960FB6F894ED
:101E7000DEBF0FBECDBFDF91CF911F910F91FF90BD
:101E8000EF90DF90CF90BF90089503E0F70142817B
:101E9000538160817181C6010E94680C29834B8344
:101EA000F701858196810E94EE0ED82EF70185817B
:101EB00096810E94EE0EC82EF701858196810E94C0
:101EC000F40E182F85E0B82E8C2D6B2D0E949D23CB
:101ED000180FF701858196810E94EE0E482F8D2DF7
:101EE0006B2D0E949D23480F2AE08C2D622F0E94AB
:101EF0009D233B81381B8D2D0E949D239981212F8D
:101F0000632F981B892F0E94AE05AFCFFC0188E09C
:101F1000808389E0818387E0828386E0838384E015
:101F2000848382E0858381E186830895FF920F9305
:101F30001F93CF93DF93EC018C01095F1F4FFF24A8
:101F4000FA9462E088810E943A2188810E94A4214B
:101F50002F81892B81F42F5F2F8360E088810E947D
:101F60003A212196C017D10761F7DF91CF911F91D8
:101F70000F91FF9008952223A1F32F3F11F41F82A8
:101F8000ECCFFF82EACFFC01E60FF11D81E09781E3
:101F9000913009F080E00895FC01E60FF11D81E029
:101FA00097819F3F09F080E00895860F911DFC0105
:101FB0008781423038F49FEF980F81E09E3F50F0C8
:101FC00080E008C08F3FE1F3642F0E949D2381E0F1
:101FD0009130B1F70895860F911DFC0187818F3FE5
:101FE00009F480E008958EBD0DB407FEFDCF8EB5D7
:101FF00008951F93CF93DF93EC01162FF89460E0C0
:102000008F850E947621888918161CF460E00E9452
:102010007621812F0E94F30F888918161CF461E045
:102020000E9476217894DF91CF911F910895E8E97D
:10203000F5E028EF31E0DF01A9011D924150504049
:10204000E1F7DC0119961C9219971A961C920895D3
:10205000CF92DF92EF92FF920F931F93CF93DF9374
:10206000EC018C858F5F8C8788E9E82E85E0F82E5F
:1020700010E0612F6064CE010E94F90F60E8CE018C
:102080000E94F90F61E08F850E94762188891816D9
:102090001CF460E00E947621670104E5F60181915D
:1020A0006F010E94F30F0150C9F7888918161CF4BC
:1020B00061E00E9476211F5FF4E5EF0EF11C1630FF
:1020C000C1F660E4CE01DF91CF911F910F91FF9097
:1020D000EF90DF90CF900C94F90FFC0160A361A307
:1020E0000895FC0160A341A30895EF92FF920F931E
:1020F0001F93CF93DF938C01D62FF42EE22EC0E0F6
:10210000CE1544F44F2D4C0F6D2FC8010E94BC0416
:10211000CF5FF6CFDF91CF911F910F91FF90EF909E
:102120000895EF92FF920F931F93CF93DF938C014B
:10213000F62ED42FE22EC0E0CE1544F46F2D6C0F96
:102140004D2FC8010E94BC04CF5FF6CFDF91CF9125
:102150001F910F91FF90EF900895EF92FF920F93D0
:102160001F93CF93DF937C01162FD42FC22F0E9491
:1021700091104FEF400F4D0F2C2F612FC7010E9480
:102180009110202F4D2F612FC7010E9475106FEF06
:102190006C0F610F202F4D2FC701DF91CF911F9141
:1021A0000F91FF90EF900C947510DF92EF92FF92D9
:1021B0000F931F93CF93DF937C01D62FD22EC42F82
:1021C000002E000C110B040F111D47FD1A958C2FCA
:1021D0000C2E000C990B8017910744F42D2D4C2FD9
:1021E0006D2FC7010E949110CF5FF1CFDF91CF918A
:1021F0001F910F91FF90EF90DF9008959F92AF9203
:10220000BF92CF92DF92EF92FF920F931F93CF93E3
:10221000DF938C01E62EF42EC22F81E0D82ED21A45
:10222000C22EC194CC0C422F4F0DC8010E94BC0499
:102230004F2D4C1B6E2DC8010E94BC046C2F6E0DDF
:102240004F2DC8010E94BC046E2D6C1B4F2DC80180
:102250000E94BC04D0E0DC170CF044C0D7FC04C0E2
:10226000C150C394C394DC0CDF5F8D2F880F8F5F48
:10227000D80E9E2C9D0EBF2CBC0E4B2D692DC80177
:102280000E94BC04AE2CAD1A4B2D6A2DC8010E94D1
:10229000BC04BF2CBC1A4B2D692DC8010E94BC0484
:1022A0004B2D6A2DC8010E94BC04BF2CBD0E4B2DC6
:1022B000AE2CAC0E6A2DC8010E94BC044B2DBE2C66
:1022C000BC1A6B2DC8010E94BC049F2C9D1A492D7D
:1022D0006A2DC8010E94BC04492D6B2DC8010E94C3
:1022E000BC04B9CFDF91CF911F910F91FF90EF9078
:1022F000DF90CF90BF90AF909F9008958F929F9264
:10230000AF92BF92CF92DF92EF92FF920F931F9303
:10231000CF93DF937C01162FD42EC22F81E0C82EDD
:10232000C21AB22EB194BB0CD0E0802F8470A82EBC
:10233000802F8270982E802F8870882E0170DC1775
:102340000CF04DC0C7FC04C0C150B394B394CB0C87
:10235000DF5F8D2F880F8F5FC80EAA2071F04D2D83
:102360004C0F612F6D0FC7010E94BC044D2D4D0F06
:102370006C2F610FC7010E94BC04992071F04D2D94
:102380004C1B612F6D0FC7010E94BC044D2D4D1BCE
:102390006C2F610FC7010E94BC04882071F04D2D85
:1023A0004D0F612F6C1BC7010E94BC044D2D4C0FBB
:1023B000612F6D1BC7010E94BC04002309F4BFCF2D
:1023C0004D2D4D1B612F6C1BC7010E94BC044D2D70
:1023D0004C1B612F6D1BC7010E94BC04B0CFDF9165
:1023E000CF911F910F91FF90EF90DF90CF90BF9012
:1023F000AF909F908F9008957F928F929F92AF920F
:10240000BF92CF92DF92EF92FF920F931F93CF93E1
:10241000DF935C01C62E942EC22F11E0121BD22E28
:10242000D194DD0C83E0F82ED0E0802F8170782EDF
:10243000882483948E0C0270DC17ACF517FD04C061
:10244000C150D394D3941D0DDF5F1F0D772099F0F9
:102450002C2F220F280D492D4C1B6C2D6D0FC50103
:102460000E9475102E2D2F0D492D4D1B6C2F6C0DBC
:10247000C5010E947510002399F02C2F220F280D02
:10248000492D4C1B6C2D6D1BC5010E9475102E2D06
:102490002F0D492D4D1B6C2D6C1BC5010E94751015
:1024A000F394F394C9CFDF91CF911F910F91FF90D7
:1024B000EF90DF90CF90BF90AF909F908F907F90E4
:1024C00008959F92AF92BF92CF92DF92EF92FF92C8
:1024D0000F931F93CF93DF93EC01B62E142FD22EC0
:1024E000AE2CAA0C922E9A18CE2CC60E292D6C2D2D
:1024F0000E949110FF24FA94F00EF10E292D4F2D19
:102500006C2DCE010E9491100A191E0D202F412F13
:102510006B2DCE010E947510DB0C6FEF6D0D202F1F
:10252000412FCE010E94751001E02E2D412F6C2D00
:10253000CE010E947E118E2D8095D80E02E02E2DA8
:10254000412F6D2DCE010E947E11FE1804E02E2D2C
:102550004F2D6D2DCE010E947E1108E02E2D4F2DA6
:102560006C2DCE010E947E11DF91CF911F910F91B2
:10257000FF90EF90DF90CF90BF90AF909F90089525
:10258000AF92BF92CF92DF92EF92FF920F931F9381
:10259000CF93DF936C01C62FF42EA22ED02F1E2DC9
:1025A000EE0CB12EB60E2E196B2D0E94D510D15007
:1025B000DE19F10E6FEF6C0F6A0D611BED2E01E05D
:1025C000212F4F2DC6010E94FC1102E0212F4F2D1B
:1025D0006B2DC6010E94FC11DF91CF911F910F91CD
:1025E000FF90EF90DF90CF90BF90AF9008952F9223
:1025F0003F925F926F927F928F929F92AF92BF9223
:10260000CF92DF92EF92FF920F931F93CF93DF93BE
:10261000EC01F901E4903196849164350CF015C118
:102620000E2C000CFF08062F062E000C110BF701D4
:10263000E00FF11F1E161F060CF007C140330CF00F
:1026400004C1A82FC42E042E000CDD085601A80ECC
:10265000B11C87FDBA941A141B040CF0F6C02E5F4F
:102660003F4F570197E0A90EB11CB7FE04C05701B8
:10267000BEE0AB0EB11CB3E0B594A794BA95E1F7F8
:1026800047FF0AC0A42FA80FAC9CC001AD9C900DC1
:102690001124281B390B40E08A2F0A2E000C990BBD
:1026A000840F911D47FD9A95C19714F0A0E3A41BD8
:1026B000F8A067FD60E0E535F10514F0E4E5F0E031
:1026C0009E2FCC85C427C62E062E000CDD08F601F1
:1026D000E01BF10B8F014F01F7E08F229924E0E816
:1026E000F0E002C0F595E7958A94E2F77E2F17FF98
:1026F00002C0095F1F4FF3E015950795FA95E1F7C2
:10270000200F311F542F577081E001C0880F5A9558
:10271000EAF7459545954595F601B4E54B02E00D80
:10272000F11D1124AF0148565A4FD0E02A2EAA0FAE
:102730003308EE24E394BB24D21513040CF085C0B7
:10274000F9015490F1E0FF121AC06901962E8A0136
:10275000E72F991608F057C08E2E852021F0D8015A
:102760008C90882A8C92E69531F4BFEFCB1ADB0A65
:10277000F6015490E0E893940F5F1F4FEACFF110F9
:102780001CC0782E70946901962E8A01E72F991645
:1027900008F039C08E2E852021F0D8018C9087203A
:1027A0008C92E69531F4BFEFCB1ADB0AF601549018
:1027B000E0E893940F5F1F4FEACFF3E0FF122CC0C5
:1027C000782E70946901862E8A01972E8916D0F48E
:1027D000E92DE52141F0D801EC916C2E682460FED2
:1027E0000FC0E82BEC93969439F4BFEFCB1ADB0AB9
:1027F000F6015490E0E89E2E83940F5F1F4FE6CFC2
:10280000E721F0CFCE25880F19F44C5A5F4F81E0B5
:10281000DF5F2A0D3B1D90CF6901962E8A01E72FBD
:10282000991688F78E2E852021F0D8018C90882665
:102830008C92E69531F4BFEFCB1ADB0AF601549087
:10284000E0E893940F5F1F4FEBCFDF91CF911F9183
:102850000F91FF90EF90DF90CF90BF90AF909F903F
:102860008F907F906F905F903F902F9008952F9260
:102870003F924F925F926F927F928F929F92AF9210
:10288000BF92CF92DF92EF92FF920F931F93CF935D
:10289000DF9300D000D000D01F92CDB7DEB74C013F
:1028A000462E342E69018E2D01111DC0E1101BC072
:1028B000C40127960FB6F894DEBF0FBECDBFDF91DF
:1028C000CF911F910F91FF90EF90DF90CF90BF902D
:1028D000AF909F908F907F906F905F904F903F90C0
:1028E0002F900C94F712F60154903196E490A52C99
:1028F000B12C9501295F3F4FA90133E055954795CC
:102900003A95E1F75B834A830370F12CEE2DF0E0FA
:10291000FD83EC835A941FEF1E0D2F2D0F2C000CFE
:10292000330B2A153B050CF070C0F982F7FE03C08B
:10293000F7E0FF0DF98329812595259525952983B4
:102940009F2D977897FF03C09150986F9F5F20E865
:10295000622E712C02C0759467949A95E2F7212C2F
:102960004981042E000C550B4E5F5F4F5F834E83F1
:10297000222D022C000C330BEC81FD812E173F071A
:102980000CF041C04A815B81429FF001439FF00DF2
:10299000529FF00D11242E813F81E20FF31FEC0DA9
:1029A000FD1DE491F0E0E621F721EF2B41F102302B
:1029B00069F0612F62194F2D033061F0452D4F19D9
:1029C000622D013039F0422D6F2D04C0652D6F1935
:1029D000412F42198823A9F0382F3370398380FFA3
:1029E00003C0552D561B652F81FF03C08E2D841B00
:1029F000482F640D430DC4010E94BC0489812394B7
:102A0000B7CF1982F6CFF39488CF27960FB6F894F4
:102A1000DEBF0FBECDBFDF91CF911F910F91FF9011
:102A2000EF90DF90CF90BF90AF909F908F907F906E
:102A30006F905F904F903F902F900895DC01FB01C5
:102A400084918F5F14968C9314973196E491EF5F85
:102A50001596EC9315976E5F7F4F5F967C936E9300
:102A60005E970895EF920F93CF93DF93EC014E871B
:102A70006D872F87E98A088B81E0888788A319A250
:102A80008F8366E273E0CE010E941E150E945A23D6
:102A900081E00E94702385E00E947E238CE00E94EA
:102AA000792361E08E850E943A2161E08D850E9444
:102AB0003A2161E08F850E943A21898918161CF419
:102AC00061E00E943A21888918161CF461E00E9496
:102AD0003A21898918166CF460E00E9476216AE038
:102AE00070E080E090E00E94382061E089890E94D7
:102AF00076218D85082E000C990BFC01E65CF94FC0
:102B0000E491F0E0EE0FFF1FE85AF94F2591349160
:102B10003D8B2C8BFC01EA5DF94FE491EB8F8E85A8
:102B2000082E000C990BFC01E65CF94FE491F0E0F3
:102B3000EE0FFF1FE85AF94F259134913B8B2A8BFA
:102B4000FC01EA5DF94FE491EA8F8889082E000CB8
:102B5000990BFC01E65CF94FE491F0E0EE0FFF1FEA
:102B6000E85AF94F259134913F8B2E8BFC01EA5D99
:102B7000F94FE491EC8F8F85082E000C990BFC0126
:102B8000E65CF94FE491F0E0EE0FFF1FE85AF94FD1
:102B900025913491398F288FFC01EA5DF94FE4913A
:102BA000ED8F61E2CE010E94F90F64E1CE010E9437
:102BB000F90F8B8587FF02C08FE78B876B85606875
:102BC000CE010E94F90F60E2CE010E94F90F6CE085
:102BD000CE010E94F90FCE01DF91CF910F91EF90BE
:102BE0000C9428104F925F926F927F928F929F92D7
:102BF000AF92BF92CF92DF92EF92FF920F931F930B
:102C0000CF93DF93EC01862EF42E102F83E58617E9
:102C10000CF485C08FE284170CF481C04C814150C4
:102C2000550B049FC001059F900D1124860F911D27
:102C300067FD9A95181619060CF071C03D818F2D0D
:102C40000F2C000C990B039F800D911D1124181659
:102C500019060CF064C078A0E62E912CC22ED12C5F
:102C6000292D092C000C330B8C8190E02817390793
:102C70000CF054C00197E0E02817390771F0C89EA6
:102C8000F001C99EF00DD89EF00D11242E0F3F1FAC
:102C9000EE8DFF8DE20FF31FE4915F2C612C492C28
:102CA000480C2D81862D062C000C990B281719062F
:102CB00091F18CF1AE2EB12CE0FF16C0113061F411
:102CC000462D4F0D642DCE010E94BC04F501F595F3
:102CD000E7956394510EE5CF012F212F452D6E2DE1
:102CE000CE010E94D510F2CF89A198A1891771F366
:102CF00088A3113041F4462D4F0D642DCE010E9462
:102D0000BC0478A2E3CF012F212F452D6E2DCE01DB
:102D10000E94D510F6CF9394E10EA2CF78A2DF9156
:102D2000CF911F910F91FF90EF90DF90CF90BF90C8
:102D3000AF909F908F907F906F905F904F9008958D
:102D40000F93CF93DF93EC01262F6A3049F4288547
:102D50009D818A85299F800D11248A8719861DC02F
:102D60006D30D9F008854A8569850E94F21528855D
:102D70003C818985239F800D112489879F81992318
:102D800061F0082E000C990B44E550E0239F401998
:102D90005109112448175907DCF281E090E0DF91D6
:102DA000CF910F910895FC01EC57FF4F7183608321
:102DB0008A579F4F445FFC01408308956F927F9232
:102DC0008F929F92AF92BF92CF92DF92EF920F932A
:102DD000CF93DF934C015C0186E8A80EB11CD501AE
:102DE0008C91882309F44AC0CCE0C81B8C3008F0D1
:102DF000C0E0F401EA5AFF4F81E080836401BEE441
:102E0000CB0ED11C60E0C6010E946D103401E3E5D9
:102E10006E0E711CD3018C9103E0080FDDE24D2F83
:102E2000481B4C0F83E0E82E24E560E0C6010E94B9
:102E3000C01261E0C6010E946D10F301808103E0C1
:102E4000080F4D2F481B4C0F24E560E0C6010E947F
:102E50006112F401E95AFF4F84E080833196D30177
:102E60008C91C81BC15DC083BC9660817181C60115
:102E70000E940422F501808181508083DF91CF91EF
:102E80000F91EF90DF90CF90BF90AF909F908F9079
:102E90007F906F900895CF92DF92FF920F931F93D0
:102EA000CF93DF93EC018C8D9D8D892B01F18E01E9
:102EB000025B1F4F40E061E0C8010E947110FE01FB
:102EC000E95AFF4FDE01AE5ABF4F9C9185E5891B41
:102ED000808331961082698D613009F46DC078F07D
:102EE000888D653008F082C06B5F811175C0DF91FD
:102EF000CF911F910F91FF90DF90CF900895CE0159
:102F000085960E94A51E81E0FE01EA5AFF4F80834C
:102F100066E273E0C8010E941E151D8E1C8EFE0124
:102F2000EC5AFF4F108288EAF82E6E018AE0C80E34
:102F3000D11CCE010E94FB178823D9F365E175E00F
:102F4000C8010E9404226A8D7B8D4AE050E0C801CE
:102F50000E94132360E075E0C8010E9404226F2DD7
:102F600062956F7070E04AE050E0C8010E94FF2255
:102F700065EF74E0C8010E94042264E0C6010E946B
:102F8000C30F8111B4CFFA94F110D3CF60E0CE011A
:102F90000E94181F83B7817F846083BF83B78160DD
:102FA00083BF83B7816083BF889583B78E7F83BFDC
:102FB00083B78E7F83BFBDCFCF58DF4F8881998184
:102FC000AA81BB818F709927AA27BB2767E0089742
:102FD000A105B10508F068E7C801DF91CF911F9105
:102FE0000F91FF90DF90CF900C942F22882309F44B
:102FF0007ECF6FE2F1CF8F929F92AF92BF92CF922E
:10300000DF92EF92FF920F931F93CF93DF93EC0128
:103010007C0180E8E80EF11CF70180809180A2809D
:10302000B3800E940720861A970AA80AB90A6E017F
:10303000FFE7CF0ED11CF601808190E0B0E0A0E068
:103040008E0105581F4F88159905AA05BB0508F084
:103050004AC0F80180819181A281B381892B8A2B9A
:103060008B2B09F440C00E940720F6012081620FDB
:10307000711D811D911DF70160837183828393838C
:103080003F9780819181A281B3810196A11DB11DDD
:1030900080839183A283B383F8011082118212820C
:1030A00013820E941320FE01E958FF4F6083718351
:1030B00082839383CE010E941C1FCE010A960E9438
:1030C000960FCE0148960E94851F81E0DF91CF9137
:1030D0001F910F91FF90EF90DF90CF90BF90AF9036
:1030E0009F908F900895F80180819181A281B38192
:1030F000892B8A2B8B2BA9F57E01F5E2EF0EF11CB3
:10310000C7010E94601DC7010E94D31DC7010E9414
:10311000971ECE010E94DE16CE010E944B177E0143
:103120008EE4E80EF11CC7010E942810FE01EC5A43
:10313000FF4F8081811103C0C7010E9417100E94B8
:103140001320F8016083718382839383FE01EB581F
:10315000FF4FC958DF4F28813981621B730B718380
:10316000608380E0B3CF2F923F924F925F926F9235
:103170007F928F929F92AF92BF92CF92DF92EF9207
:10318000FF920F931F93CF93DF93CDB7DEB7659771
:103190000FB6F894DEBF0FBECDBF6C016A8B7B8B80
:1031A0004B83FC01EC5AFF4F10822FEF2D831C82C2
:1031B0001D8A10E31C8A3C013AE0630E711C842FC7
:1031C00090E09F838E832601E3E54E0E511C46015D
:1031D000F5E28F0E911C9601295A3F4F39872887B7
:1031E000C601885A9F4F9B878A87F601EA5AFF4F8C
:1031F000FF87EE8722503109398B288B0A971C01F3
:10320000C6010E94FB178823D9F364E0C3010E9422
:10321000C30F012F110F110B882399F0F201F081D8
:10322000F1952B81F29F202D112422502D8B64E0EB
:10323000C3010E94C30F811193C0C4010E94001FEB
:1032400094C065E0C3010E94C30F8111E7CF66E01F
:10325000C3010E94C30F8111E1CF8C81811185C010
:1032600044E063E0C3010E94D50F882331F09C89BC
:103270009F5F9C8BC4010E94041F44E061E0C30176
:103280000E94D50F882331F0EC89E150EC8BC4010A
:103290000E94041FFC898F2F0F2E000C990B2E818A
:1032A0003F818217930709F46BC0F7FF03C03B818E
:1032B00031503C8BF2018081F4E0F80F2C89829F21
:1032C000F0191124FD8B9D89090F111D97FD1A9589
:1032D00017FF02C00F5F1F4FF801F595E795FA83BE
:1032E000E9830981102FE885F9851082EA85FB853D
:1032F000008321E0EE85FF852083E889F98910822B
:10330000EA88FB88B12CA12C2C89022E000C330BEF
:103310003D872C878E819F818A159B0599F1EC85CD
:10332000FD85EA15FB0579F423E0E885F98520831E
:10333000F2018081F02F2C89289FF00D11248F2F0E
:10334000EA85FB858083F70165917491C1010E9434
:103350004A22FFEFAF1ABF0A22E0E20EF11CDACFD9
:10336000C4010E94FC1E3C893D83C8013D89831B2A
:10337000910937FD9395029764F181E08C83A3CF87
:103380001C8A98CF60E0C1010E946D10F20180811B
:103390004981FC89F89F400D1124415024E560E0EB
:1033A000C1010E94911061E0C1010E946D10F20103
:1033B000808103E0080F4981FC898F9F400D112413
:1033C000425083E0E82E24E560E0C1010E946112D2
:1033D00017CF8D8165960FB6F894DEBF0FBECDBFB7
:1033E000DF91CF911F910F91FF90EF90DF90CF90E1
:1033F000BF90AF909F908F907F906F905F904F9015
:103400003F902F9008950F931F93CF93DF93EC017C
:103410008C01025B1F4FC8010E9417106DEC74E015
:10342000C8010E940422C8010E94281083E00E9463
:103430007E2389E491E0EEEFFFE30995FE01EC5A6B
:10344000FF4F108268EA74E0C8010E944A22C80156
:103450000E9428102A96CE010E94960F64E0CE01A9
:103460000E94C30F811107C062E370E080E090E02A
:103470000E943820F0CFDF91CF911F910F910895D6
:103480002F923F924F925F926F927F928F929F9274
:10349000AF92BF92CF92DF92EF92FF920F931F9362
:1034A000CF93DF93CDB7DEB729970FB6F894DEBF81
:1034B0000FBECDBF998788877B836A832A013C0131
:1034C00080E7680E711CF3018081882309F4F7C03E
:1034D00081E0E885F985EA5AFF4F8083E885F98520
:1034E000EB5AFF4F1082E885F985EC5AFF4F1082A6
:1034F000E885F985108E8F01025B1F4F61E0C801DE
:103500000E946D10888599858D5A9F4F9F838E8369
:10351000A884B98497E5A90EB11CE884F984E8E58C
:10352000EE0EF11C88849984F2E58F0E911C88853B
:1035300099858F589F4F9D838C83288439849AE086
:10354000290E311CC884D984E5E2CE0ED11C8885B1
:1035500099850E94FB178823D1F3EA81FB81F491BE
:10356000F983FF2321F0EE81FF81F081F98327E3C6
:1035700035E040E060E0C8010E94F71241145104B8
:1035800039F04981445F920160E0C8010E94F7125E
:10359000F50110828CE0F70180836A817B81C8018C
:1035A0000E940422F4018081982F990F990F891BA2
:1035B0008D5AF5018083EE81FF818081982F990FCC
:1035C000990F891B835DF7018083EC81FD818081E8
:1035D00063E375E084FD02C06FE275E0C8010E94FC
:1035E0004A22F4018081982F990F990F891B8D5AD7
:1035F000F5018083F70180818F5F8083E885F985FD
:1036000082A56BE275E0811102C067E275E0C80136
:103610000E944A22F4018081982F990F990F891BEB
:103620008D5AF5018083F70180818F5F808363E28B
:1036300075E0C8010E944A2265E0C1010E94C30FE3
:10364000882351F0E885F98562A56F5FC6010E9465
:10365000081FC6010E94041F64E0C1010E94C30F3D
:1036600081111FC0F3012081422F50E070E060E023
:10367000EC81FD8180819181A281B38184179507BE
:10368000A607B70710F02F3F61F466E0C1010E9462
:10369000C30F882309F45BCF888599850E94031A9C
:1036A00056CF8FEFF301808360E0C6010E949A1E1F
:1036B000C6010E94FC1E81E0E885F985808F29966D
:1036C0000FB6F894DEBF0FBECDBFDF91CF911F9133
:1036D0000F91FF90EF90DF90CF90BF90AF909F90B1
:1036E0008F907F906F905F904F903F902F900895B4
:1036F00050E040E00C94401AE0E8F7E7259134915F
:1037000081E02130304C09F080E00895CF93DF93C1
:10371000EC010E947C1B9E01275A3F4FDE01A059FD
:10372000BF4F882309F440C0E6E9F7E78491F90127
:103730008083E7E9F7E7E491EC83E8E9F7E7E491D0
:10374000ED83E9E9F7E7859194919F838E83EBE917
:10375000F7E78591949199878887EDE9F7E7E491F8
:10376000EBA7EEE9F7E7E491EAA7EFE9F7E7E491E1
:10377000EC93E0EAF7E7859194919D8F8C8FE2EAD4
:10378000F7E7859194919F8F8E8FE4EAF7E7859113
:10379000949199A388A3E6EAF7E7859194919BA376
:1037A0008AA3DF91CF9108958CE3F90180831C8275
:1037B0008FEF8D8320E233E03F832E8324ED33E0CF
:1037C0003987288791E09BA79AA78C938CEA9DE084
:1037D0009D8F8C8F8EED9DE09F8F8E8F84E79EE076
:1037E00099A388A38CE39FE0DACFCF92DF92EF9288
:1037F0000F93CF93DF93EC01FC01E158FF4F82E37D
:103800008083349781E090E0A0E0B0E080839183F2
:10381000A283B3833B978FEF8083CE010E94861BE8
:10382000CE010E94141F6FEFCE010E94181F6E017F
:103830008AE0C80ED11CC6010E94860FC6010E94F4
:10384000960FCE0148960E947B1F8EE0E82E0FE077
:1038500020E14BE06DE0CE01825B9F4F0E9432156C
:10386000A596CE010E94991C65E0C6010E94C30F77
:10387000882351F060E0CE01DF91CF910F91EF905E
:10388000DF90CF900C94081F40E067EA75E0CE010E
:10389000DF91CF910F91EF90DF90CF900C942D1D81
:1038A000CF93DF93D62FC72F0E947C1B882359F01C
:1038B000AD2FBC2FEBE8F7E784918D933196E53976
:1038C00087E7F807C9F7DF91CF910895CF93DF938A
:1038D000DC0170E0660F771F1F96ED91FC91509709
:1038E000E60FF71F2591349190963C932E935F97A6
:1038F000F9014591549114968C911497849F402D11
:10390000112491964C939197F901C591D4916D2F03
:1039100070E04617170629F020F0F901259134913F
:10392000432F849F402D112492964C93DF91CF9189
:10393000089521E0FC01248324E020A726E036E05E
:10394000308B278760E00E94661C61E070E083E0B6
:103950000E94B420E1EBF0E08081887F8160808369
:10396000F89410928000E1E8F0E010821092850057
:103970001092840088E191E0909389008093880000
:10398000808188608083808181608083EFE6F0E0C1
:10399000808182608083789408950F93FC010111E7
:1039A00007C06230D9F030F4662379F0613091F0CD
:1039B0000F9108956330C9F06430D1F76481649F3A
:1039C000402D1124458F268FF3CF4B3008F04AE06D
:1039D000468BEECF642F0F910C94661C6481649F1C
:1039E000402D1124418F228FE3CF6481649F402DAD
:1039F0001124438F248FDCCF80919C07882329F0EA
:103A0000809199078093B400089580E0FBCFFC017A
:103A1000178A158A14A213A2108E10929907109279
:103A20009A0710929C070C94FC1C0F931F93CF9342
:103A3000DF93EC018B010E94071D1E870D871B8AF7
:103A40001A8A81E0898389E08E8B198E1B8E1D8EE8
:103A5000DF91CF911F910F910895411102C00C94F5
:103A6000151D0895CF93DF93EC01611115C0888176
:103A7000882391F0898181110FC0E9858E2F90E014
:103A8000880F991FEF81F885E80FF91F85919491B0
:103A90008F3F980721F41882DF91CF9108959C877A
:103AA0009927880F991FEA85FB85E80FF91F659113
:103AB0007491CE010E94151D89858F5F8987ECCF97
:103AC00060E00C94321D0F93CF93DF93EC016111F2
:103AD00066C08981882309F462C08D8981115FC025
:103AE0008D859E85EA89FB89EE0FFF1FE80FF91F80
:103AF000459154914115510541F42989213021F511
:103B00001B8A1A8AFC0145915491BA0176956795F2
:103B100076956795862F40FF2EC0252F26952695F2
:103B20002695205186E0569547958A95E1F74F7185
:103B30006F7000E0CE010E94CD1CEA89FB893196AE
:103B4000FB8BEA8BCF010AC019828881882369F038
:103B500060E0CE010E94321D8A899B89880F991FDF
:103B6000ED85FE85E80FF91FCECFCE01DF91CF9115
:103B70000F910C94071D8F738C8B8C81859F802DEA
:103B800011248D8B1DA21CA21BA281E08F8B809320
:103B90009C07188E8A899B8901969B8B8A8BDF9163
:103BA000CF910F91089560E00C94631DCF93DF9344
:103BB000EC016111B3C08F89882309F4AFC08D89EE
:103BC000811105C0CE01DF91CF910C94071D81506A
:103BD0008D8B8DA1811134C02BA13CA12F5F3F4F54
:103BE000C901880F991FEF8DF8A1E80FF91F859182
:103BF0009491482F47704EA3492F469546954FA361
:103C0000AC0164E0569547956A95E1F74F739C8146
:103C1000499F402D11244DA383FB882780F9809371
:103C200098073CA32BA389A190E02817390740F0FF
:103C30002AA1222309F475C0821B91099CA38BA39E
:103C40008DA181508DA3888D31E0380F388F4C893C
:103C50002FA1240F8C85280F2A836B8D662361F09A
:103C600070E0832F032E000C990B0E94BD238C8DD6
:103C7000869F200D11242A838A8190E0CB966BE3E6
:103C800070E00E94BD238A832E892B83698D662371
:103C900071F0062E000C770B832F032E000C990B6E
:103CA0000E94BD238A8D869F200D11242B836D8D4C
:103CB000662389F0832F330F990B70E00E94BD2398
:103CC000CB0162E070E00E94BD232E8D9B81289F76
:103CD000900D11249B834F3341F18B818A300CF07E
:103CE00089E087FD80E08B83F894EA81F0E0EB5473
:103CF000FA4FE491E0939B078D8198A5899F802DD1
:103D000011249B81899F802D11249EA1899F802D44
:103D1000112480939A07809399077894DF91CF912B
:103D20000895CE010E94071D8BCF1B82DDCF60E07E
:103D30000C94D61DCF93DF93EC01611103C00E9458
:103D4000071D1982DF91CF910895CF93DF93EC0186
:103D50000E94071D1982DF91CF91089560919A0703
:103D6000662329F180919D078F5F80939D07909135
:103D70009B078917E0F081E090919C07911180E00A
:103D800080939C0710929D0780919807882369F083
:103D90008091040193E4899F802D1124895B809395
:103DA00004010E949D23909399070C94FC1C089594
:103DB0001F920F920FB60F9211242F933F934F93A0
:103DC0005F936F937F938F939F93AF93BF93EF9383
:103DD000FF930E94AE1EFF91EF91BF91AF919F9113
:103DE0008F917F916F915F914F913F912F910F90A4
:103DF0000FBE0F901F9018956EEF75E00C94151D77
:103E000066EF75E00C94151D60EF75E00C94151DC0
:103E1000FC01862F660F990B668170E06F5F7F4F04
:103E20000E94BD238583089521E0FC01208308952D
:103E300070E085E00C94B420AF92BF92CF92DF92F5
:103E4000EF92FF920F931F93CF93DF93EC01898141
:103E50009A812FE0289F8001299F100D112485E170
:103E60000E949920800F911F24E0969587952A95AE
:103E7000E1F79A8389832881222391F1EC81AD8037
:103E8000B12CD12CC12CA885B9857D0110E000E0B2
:103E90006E817F819B0150E040E08617970728F0F4
:103EA000BC01A817B90708F4BD0190E080E01F929B
:103EB0001F921F92EF930E9419236B830F900F9014
:103EC0000F900F9070E085E0DF91CF911F910F91DF
:103ED000FF90EF90DF90CF90BF90AF900C94B42004
:103EE000DF91CF911F910F91FF90EF90DF90CF90D6
:103EF000BF90AF900895FC018CE39FE09383828391
:103F000084E0818381E084870895CF93DF93EC017F
:103F10008C819D81892B21F18C858F7139F584E10C
:103F20000E949920BC01990F880B990B0E946F2465
:103F300026EE3FE34EEC50E40E94FB240E943E2418
:103F40009B017B836A83672BA9F084E08983FE0150
:103F5000349680E0419151912417350720F48983EC
:103F6000DF91CF9108958F5F8430A1F78C858F5FAB
:103F70008C87F6CF8FEF8983F9CF1F920F920FB600
:103F80000F9211242F933F938F939F93AF93BF93DF
:103F900080919F079091A007A091A107B091A207DF
:103FA00030919E0723E0230F2D3758F50196A11D70
:103FB000B11D20939E0780939F079093A007A09325
:103FC000A107B093A2078091A3079091A407A091A5
:103FD000A507B091A6070196A11DB11D8093A30767
:103FE0009093A407A093A507B093A607BF91AF91A4
:103FF0009F918F913F912F910F900FBE0F901F9027
:10400000189526E8230F0296A11DB11DD2CF2FB718
:10401000F89460919F077091A0078091A1079091FB
:10402000A2072FBF08953FB7F8948091A3079091FE
:10403000A407A091A507B091A60726B5A89B05C027
:104040002F3F19F00196A11DB11D3FBFBA2FA92F17
:10405000982F8827BC01CD01620F711D811D911D14
:1040600042E0660F771F881F991F4A95D1F7089580
:10407000CF92DF92EF92FF92CF93DF936B017C019F
:104080000E941320EB01C114D104E104F10439F4BE
:10409000DF91CF91FF90EF90DF90CF9008950E9435
:1040A00013206C1B7D0B683E734068F381E0C81AD7
:1040B000D108E108F108C851DC4FE5CF789484B508
:1040C000826084BD84B5816084BD85B5826085BD14
:1040D00085B5816085BDEEE6F0E0808181608083FA
:1040E000E1E8F0E0108280818260808380818160DD
:1040F0008083E0E8F0E0808181608083E1EBF0E0A4
:10410000808184608083E0EBF0E080818160808347
:10411000EAE7F0E080818460808380818260808330
:104120008081816080838081806880831092C1005B
:1041300008958E3008F08E502091050190E4299F5B
:10414000900111248770822B80937C0080917A00EB
:10415000806480937A0080917A0086FDFCCF809104
:1041600078009091790008951F93CF93DF93182FD3
:10417000EB0161E00E943A21209739F460E0812F41
:10418000DF91CF911F910C947621CF3FD10511F48F
:1041900061E0F5CFE12FF0E0EE5EF94FE491E3301E
:1041A00031F140F4E130B1F0E230E1F0C038D10556
:1041B0007CF7E4CFE63029F1E73059F1E430B1F78C
:1041C00080918000806280938000D0938B00C093A8
:1041D0008A0004C084B5806884BDC7BDDF91CF91DB
:1041E0001F91089584B5806284BDC8BDF7CF8091CA
:1041F0008000806880938000D0938900C0938800FD
:10420000EDCF8091B00080688093B000C093B30080
:10421000E5CF8091B00080628093B000C093B4007D
:10422000DDCF833081F028F4813099F08230A9F01D
:1042300008958630A9F08730C9F08430B1F48091B8
:1042400080008F7D03C0809180008F7780938000F5
:10425000089584B58F7784BD089584B58F7DFBCF95
:104260008091B0008F778093B00008958091B00066
:104270008F7DF9CFCF93DF9390E0FC01EA5DF94F9A
:104280002491865C994FFC0184918823C9F090E0C9
:10429000880F991FFC01EE59F94FA591B491FC01CB
:1042A000E85AF94FC591D49161110DC09FB7F894A8
:1042B0008C91209582238C938881282328839FBF0B
:1042C000DF91CF910895623051F49FB7F8943C91FB
:1042D000822F809583238C93E8812E2BEFCF8FB78D
:1042E000F894EC912E2B2C938FBFEACF1F93CF9392
:1042F000DF93162F282F30E0F901EE5EF94F8491FD
:10430000F901EA5DF94FD491F901E65CF94FC491E6
:10431000CC23A1F081110E941121EC2FF0E0EE0FCF
:10432000FF1FE85AF94FA591B4918FB7F894EC911B
:10433000111108C0D095DE23DC938FBFDF91CF91A0
:104340001F910895DE2BF8CFCF93DF93282F30E015
:10435000F901EE5EF94F8491F901EA5DF94FD491CC
:10436000F901E65CF94FC491CC23A1F081110E94C0
:104370001121EC2FF0E0EE0FFF1FE25BF94FA5914A
:10438000B491EC91ED2381E090E009F480E0DF91BD
:10439000CF91089580E090E0FACFCF92DF92EF9234
:1043A000FF920F931F93CF93DF936C01EB017B017F
:1043B000E40EF51E10E000E0CE15DF0561F0699116
:1043C000D601ED91FC910190F081E02DC601099597
:1043D000080F191FF1CFC801DF91CF911F910F91E5
:1043E000FF90EF90DF90CF900895FB0101900020A7
:1043F000E9F73197AF01461B570BDC01ED91FC91BA
:104400000280F381E02D0994EF92FF920F931F93A6
:10441000CF93DF937C018B01D0E0C0E0F801649181
:104420000F5F1F4F662359F0D701ED91FC9101906A
:10443000F081E02DC7010995C80FD91FEFCFCE013C
:10444000DF91CF911F910F91FF90EF90089561152B
:10445000710511F00C94F52190E080E00895DC01E5
:10446000ED91FC910190F081E02D09940F931F9341
:10447000CF93DF93EC016DE00E942F228C016AE064
:10448000CE010E942F22800F911FDF91CF911F91AB
:104490000F9108950F931F93CF93DF93EC010E9428
:1044A00004228C01CE010E943622800F911FDF91E1
:1044B000CF911F910F9108958F929F92AF92BF92CB
:1044C000CF92DF92EF92FF920F931F93CF93DF93E0
:1044D000CDB7DEB7A1970FB6F894DEBF0FBECDBF44
:1044E0006C01142FE52FCB01022F19A2223008F402
:1044F0000AE07E0121E2E20EF11C802E912CB12C0B
:10450000A12C612F7E2FA50194010E94D123029F2F
:10451000101911241A303CF5105DF70112937F0138
:10452000122FE32FCA01232B242B252B51F790E0C8
:1045300080E0E114F10421F0B701C6010E94F521E9
:10454000A1960FB6F894DEBF0FBECDBFDF91CF911D
:104550001F910F91FF90EF90DF90CF90BF90AF90A1
:104560009F908F900895195CD8CFCF92DF92EF92F1
:10457000FF920F931F93CF93DF93EC016A017B01AE
:104580002115310579F4E881F9810190F081E02D60
:10459000642FDF91CF911F910F91FF90EF90DF90EB
:1045A000CF9009942A303105E9F42AE0F7FE1AC0C9
:1045B0006DE20E942F228C0144275527BA014C1925
:1045C0005D096E097F092AE0CE010E945C22800FFE
:1045D000911FDF91CF911F910F91FF90EF90DF908E
:1045E000CF900895B701A601CE01DF91CF911F9121
:1045F0000F91FF90EF90DF90CF900C945C229A0186
:10460000AB01770F660B770B0C94B52221153105A2
:1046100041F4DC01ED91FC910190F081E02D642FDB
:1046200009940C945C229A01AB0170E060E00C9458
:1046300006234F925F926F927F92AF92BF92CF927A
:10464000DF92EF92FF920F931F93CF93DF93CDB73B
:10465000DEB729013A019B01AC012419350946094D
:10466000570989899A89AB89BC89BC01CD016A192E
:104670007B098C099D090E948D23A80197012419AB
:104680003509460957090E94F323CA01B9016A0D89
:104690007B1D8C1D9D1DDF91CF911F910F91FF9070
:1046A000EF90DF90CF90BF90AF907F906F905F9032
:1046B0004F90089561E08AE00E94762161E08AE0EF
:1046C0000E943A218CB580618CBD8CB580648CBD14
:1046D00061E08DE00E943A2161E08BE00C943A2188
:1046E000811104C08CB580628CBD08958CB58F7D1E
:1046F000FBCF9CB5937F892B8CBD08959CB59C7F87
:10470000282F2370922B9CBD9DB582FB222720F978
:10471000892F8E7F822B8DBD0895DB018F939F9310
:104720000E941224BF91AF91A29F800D911DA39F63
:10473000900DB29F900D11240895991B79E004C04B
:10474000991F961708F0961B881F7A95C9F78095D0
:104750000895AA1BBB1B51E107C0AA1FBB1FA617C8
:10476000B70710F0A61BB70B881F991F5A95A9F71A
:1047700080959095BC01CD01089597FB072E16F406
:10478000009407D077FD09D00E94A92307FC05D02B
:104790003EF4909581959F4F0895709561957F4F58
:1047A0000895A1E21A2EAA1BBB1BFD010DC0AA1F72
:1047B000BB1FEE1FFF1FA217B307E407F50720F08A
:1047C000A21BB30BE40BF50B661F771F881F991F05
:1047D0001A9469F760957095809590959B01AC014E
:1047E000BD01CF010895052E97FB1EF400940E9491
:1047F0000A2457FD07D00E94D12307FC03D04EF4B2
:104800000C940A2450954095309521953F4F4F4F79
:104810005F4F089590958095709561957F4F8F4F6C
:104820009F4F08950E942F24A59F900DB49F900D37
:10483000A49F800D911D112408950024A7FD0094CC
:104840002A0F301D401D501D601D701D801D901DC4
:104850000895EE0FFF1F0590F491E02D0994A29F9B
:10486000B001B39FC001A39F700D811D1124911D44
:10487000B29F700D811D1124911D08950E94DA24AC
:1048800088F09F5798F0B92F9927B751B0F0E1F011
:10489000660F771F881F991F1AF0BA95C9F714C0C1
:1048A000B13091F00E94F424B1E008950C94F42406
:1048B000672F782F8827B85F39F0B93FCCF38695FA
:1048C00077956795B395D9F73EF490958095709557
:1048D00061957F4F8F4F9F4F0895E89409C097FBD4
:1048E0003EF490958095709561957F4F8F4F9F4FC7
:1048F0009923A9F0F92F96E9BB279395F69587950B
:1049000077956795B795F111F8CFFAF4BB0F11F4CD
:1049100060FF1BC06F5F7F4F8F4F9F4F16C0882374
:1049200011F096E911C0772321F09EE8872F762FAA
:1049300005C0662371F096E8862F70E060E02AF0EB
:104940009A95660F771F881FDAF7880F96958795D7
:1049500097F9089597F99F6780E870E060E00895FF
:104960009FEF80EC089500240A9416161706180687
:104970000906089500240A94121613061406050663
:104980000895092E0394000C11F4882352F0BB0FF4
:1049900040F4BF2B11F460FF04C06F5F7F4F8F4F57
:1049A0009F4F089557FD9058440F551F59F05F3F92
:1049B00071F04795880F97FB991F61F09F3F79F041
:1049C00087950895121613061406551FF2CF4695C3
:1049D000F1DF08C0161617061806991FF1CF869545
:1049E0007105610508940895E894BB276627772729
:1049F000CB0197F908950E940E250C94C1240E94C2
:104A0000B32438F00E94BA2420F0952311F00C94BE
:104A1000AA240C94B02411240C94F5240E94D224CE
:104A200070F3959FC1F3950F50E0551F629FF00101
:104A3000729FBB27F00DB11D639FAA27F00DB11D1A
:104A4000AA1F649F6627B00DA11D661F829F2227A3
:104A5000B00DA11D621F739FB00DA11D621F839F2A
:104A6000A00D611D221F749F3327A00D611D231F00
:104A7000849F600D211D822F762F6A2F11249F574E
:104A800050409AF0F1F088234AF0EE0FFF1FBB1F51
:104A9000661F771F881F91505040A9F79E3F510510
:104AA00080F00C94AA240C94F5245F3FE4F3983E24
:104AB000D4F3869577956795B795F795E7959F5FBA
:104AC000C1F7FE2B880F911D9695879597F908954C
:104AD0008F929F92AF92BF92CF92DF92EF92FF920E
:104AE000CF93DF93EC01688179818A819B81611585
:104AF00071058105910521F464E279ED8BE597E07C
:104B00002DE133EF41E050E00E94F32349015A01C7
:104B10009B01AC01A7EAB1E40E9412246B017C0165
:104B2000ACEEB4EFA50194010E947528DC01CB0125
:104B30008C0D9D1DAE1DBF1DB7FF03C00197A109C0
:104B4000B04888839983AA83BB839F77DF91CF91F5
:104B5000FF90EF90DF90CF90BF90AF909F908F909D
:104B600008950E946825089580E091E00E946825DC
:104B70000895B0E0A0E08093000190930101A0931C
:104B80000201B09303010895AEE0B0E0EAECF5E273
:104B90000C9488280D891E898F89988D26E02C8396
:104BA0001A83098397FF02C080E090E801979E83F3
:104BB0008D83AE01455E5F4F698D7A8DCE01019682
:104BC0000E94F4254D815E8157FD0AC02F813885F2
:104BD000421753070CF49A01020F131FF8011082B9
:104BE0002E96E4E00C94A428ABE0B0E0EAEFF5E206
:104BF0000C947A287C013B018A01FC011782168201
:104C0000838181FFC8C1CE0101965C01F7019381C8
:104C1000F30193FD859193FF81913F01882309F46E
:104C200053C1853239F493FD859193FF81913F0102
:104C3000853229F4B70190E00E94E427E7CF912C58
:104C4000212C312CFFE1F31538F08B3211F190F467
:104C5000803209F1833229F137FC3CC020ED280F66
:104C60002A3050F536FE20C08AE0989E200D11248F
:104C7000922E06C08D3291F0803371F7689430F82F
:104C8000F30193FD859193FF81913F018111DACF6B
:104C900021C0689431F8689432F8F2CF689433F800
:104CA000EFCF689434F8ECCFEAE02E9E200D11246B
:104CB000222E689435F8E4CF8E3229F436FC04C1F4
:104CC000689436F8DDCF8C3619F4689437F8D8CF6D
:104CD0008836B1F2982F9F7D95549330E0F083365B
:104CE000A1F18337C1F1833509F063C02801F2E0F7
:104CF0004F0E511CF801C080D180692D70E036FC48
:104D000002C06FEF7FEFC6010E94CE274C0168946E
:104D100037F882010AC00C5F1F4FFFE3F983882434
:104D20008394912C6501E89437F833FE2DC0522C02
:104D30008114910471F5552009F468CFB70180E220
:104D400090E00E94E4275A94F6CFF801808189838D
:104D50000E5F1F4FE4CF2801F2E04F0E511CF80107
:104D6000C080D180692D70E036FC02C06FEF7FEF0C
:104D7000C6010E94D9274C018201D5CFB70180E23C
:104D800090E00E94E4272A942814190409F0B0F74F
:104D9000CECFF60137FC859137FE81916F01B701C7
:104DA00090E00E94E42751105A94F1E08F1A910884
:104DB000BFCF843619F0893609F077C0F80137FE85
:104DC0006BC060817181828193810C5F1F4FF32DD5
:104DD000FF763F2E97FF09C090958095709561955D
:104DE0007F4F8F4F9F4F689437F82AE030E0A5013E
:104DF0000E941428C82ECA188C2C432C36FE0CC0D6
:104E0000E89440F8C91440F434FE05C032FC03C0F5
:104E1000F32DFE7E4F2E892C44FE95C0FE01EC0D35
:104E2000F11D8081803309F087C0242D297E422E18
:104E3000842D8870582E43FC95C040FE8FC09C2C5A
:104E4000821418F42C0C922C981844FE91C0B701CF
:104E500080E390E00E94E42742FE09C088E790E0EA
:104E600041FE02C088E590E0B7010E94E427C91422
:104E700008F48AC0CA94D12C9FEFC91AD90ACA0C67
:104E8000DB1CF60182916F01B70190E00E94E427DC
:104E9000AC14BD04B1F74FCF60817181072E000CB7
:104EA000880B990B0E5F1F4F92CFD32CE894D4F848
:104EB0002AE030E0853739F1232D297FD22E8F3635
:104EC00001F148F48835A9F0F701868197812B9686
:104ED000E2E10C949628803749F08837A9F7D4FE90
:104EE00002C06894D2F820E130E00DC06894D4F894
:104EF000F6CF34FE03C0822F8660D82E20E132E048
:104F000002C028E030E0F801D7FE0FC06081718157
:104F1000828193810C5F1F4FA5010E941428C82E27
:104F2000CA183D2CE89437F867CF6081718190E012
:104F300080E00E5F1F4FF0CF42FC02C0839478CF19
:104F40008394839475CF842D867809F471CFF6CF3E
:104F5000B70180E290E00E94E42783948214C0F3BA
:104F6000512C73CF522C5818821408F46ECFF8CFFE
:104F7000842D867809F47BCF8BE241FE80E247FCEA
:104F80008DE2B70190E071CFB70180E390E00E941D
:104F9000E4279A946CCF8FEF9FEF99CFFC01059097
:104FA000615070400110D8F7809590958E0F9F1F2B
:104FB0000895FC016150704001900110D8F7809570
:104FC00090958E0F9F1F08950F931F93CF93DF939C
:104FD000182F092FEB018B8181FD09C01FEF0FEF07
:104FE000812F902FDF91CF911F910F91089582FF14
:104FF00014C02E813F818C819D81281739073CF494
:10500000E881F981CF0101969983888310838E818D
:105010009F8101969F838E83E3CFE885F985812F59
:105020000995892BA1F3DACFFA01AA27283051F18B
:10503000203181F1E8946F936E7F6E5F7F4F8F4FC9
:105040009F4FAF4FB1E03ED0B4E03CD0670F781F28
:10505000891F9A1FA11D680F791F8A1F911DA11D0D
:105060006A0F711D811D911DA11D20D009F4689446
:105070003F912AE0269F11243019305D3193DEF6EE
:10508000CF010895462F4770405D4193B3E00FD0A4
:10509000C9F7F6CF462F4F70405D4A3318F0495D8F
:1050A00031FD4052419302D0A9F7EACFB4E0A69572
:1050B0009795879577956795BA95C9F70097610594
:1050C000710508959B01AC010A2E069457954795EA
:1050D00037952795BA95C9F7620F731F841F951FDF
:1050E000A01D0895B7FF0C9412240E941224821B65
:1050F000930B08952F923F924F925F926F927F92FF
:105100008F929F92AF92BF92CF92DF92EF92FF92D7
:105110000F931F93CF93DF93CDB7DEB7CA1BDB0B83
:105120000FB6F894DEBF0FBECDBF09942A88398828
:1051300048885F846E847D848C849B84AA84B9842F
:10514000C884DF80EE80FD800C811B81AA81B9813B
:10515000CE0FD11D0FB6F894DEBF0FBECDBFED014F
:10516000089513E0C8E3D3E004C0FE010E9429249F
:0C5170002196C933D107C9F7F894FFCF8E
:10517C00010000000101573D256400473D256400F6
:10518C00463D25640048503D2575004261727261B0
:10519C00636B73004275696C640041747461636B7A
:1051AC00001B013E0D00000000240100002A01003C
:1051BC000000000000A016CD214C4F414445520088
:04000003000006C62D
:00000001FF
